:03000000021916CC
:0C19160078FFE4F6D8FD7581C2020036AF
:0100110022CC
:06166D008B308A31893246
:10167300756A027F4812179312196EEF20E0F9ABD7
:1016830030AA31A93212068D7872E6FE08E6FDED26
:01169300FF57
:011694002233
:100EAE0043525354005341564500434647002D3E8E
:100EBE0053320052415445434C5220554E495442F0
:100ECE004C4E4B5452455644464C54534156455243
:100EDE00535420535720202E323520317320203288
:100EEE00732020357320203130732033307320313E
:100EFE006D2020326D2020356D202031306D203355
:100F0E00306D203168202032682020346820205433
:100F1E007269670000000100040008001400280038
:100F2E007800F001E004B009601C2038407080E1C8
:100F3E0000FFFF46656574596172644D6574724FAA
:0F0F4E006666204F6E20204E6F2020596573205D
:0C19220025E02421F582E4340FF5832237
:1015180078B576AB0876CD087600087604E408F648
:1015280008760108F60876FA08764008F608F608FC
:10153800F608F67BFF7A0E79AE1215B47F05121401
:04154800AD021617C3
:1017AE00756E1D756FC01214E378B6E664CD7004C5
:0917BE0018E664AB600312151873
:0117C70022FF
:0D18DE00C2AF7DC07C1DE4FF12186AD2AFBE
:0118EB0022DA
:1014E300753FFF856E40856F4175420075430075FA
:1014F30044B5E4FFAB3FAA40A9418F827583001234
:101503000660AB42AA43A9448F8275830012069FEB
:041513000FBF0EE018
:0115170022B1
:101617007D01E4FF12173B7BFF7A0E79B31215B4F5
:101627001218DEC2AF7FB57B0E7DC07C1D12187409
:0D163700D2AF7F021214ADE4FDFF02173B9D
:100A3700E4F5307BFF7A0E79B81215B47F051214EE
:100A4700ADA297829650FAA296920FA2979210E5BE
:100A57003075F004A424C1F9740E35F0FA7BFF1247
:100A670015B47F051214AD853031E4F5327BFF7A7A
:100A77000E79BC1215B4E53024FE602B14603014D7
:100A87006035240470397F01EF12192278B7E6FC2C
:100A970008E6FD7401936D7003E4936C70028F3266
:100AA7000FBF10E4020B3A78B9E6F532020B5F7814
:100AB700BAE6F532020B7C78C1E6F532020B99E50E
:100AC700306531708AA20F309601B35013A2969207
:100AD7000F30960C0530E530C394084003E4F53039
:100AE700A210309701B350D7A29792103097D0E554
:100AF70030B4080050C9900B04F8282873020B1C67
:100B0700020B47020B4D020B6A020B87020BAD0269
:100B17000BB3020BB90532E532C3941040037532AB
:100B270001E532121922E493FF74019378B7CFF6E7
:100B370008EFF6E53275F004A424E1F9740E805B42
:100B470012116B020AC60532E532C394034003E46F
:100B5700F53278B9A632E53275F004A42441F97468
:100B67000F80380532E532C394024003E4F532784A
:100B7700BAA632E53275F004A4244DF9740F801B30
:100B87000532E532C394024003E4F53278C1A63258
:100B9700E53275F004A42455F9740F35F0FA7BFF9C
:100BA7001215B4020AC6121518020AC6121617023F
:080BB7000AC643A208020AC6A7
:0A193A004552415300444F4E450052
:10175900E4D3FCFD7B80FAF9F80207EC78B7E6F5EB
:0D1769005608E6F55722E563AE62780622C9
:10104C00C20DC20EE4F531F532AE31AF3212175982
:10105C00401CE53064816016AF32AE311215E612D9
:10106C0018568F300532E53270DF053180DBE53004
:10107C00B48108E532153270021531AE31AF32E46D
:10108C00C312175B700CD20D1218FAE4F562F563FB
:10109C008007853162853263E4F564F565755580AA
:0310AC00121765B3
:0110AF00221E
:0415E6008F828E83DF
:1015EA001217594027E582AE837806C333CE33CE2D
:1015FA00D8F9FD756A02EE7872F6CFEDCFEF08F6EC
:0C160A007F5012181412196EEF20E0F946
:0116160022B1
:0317C800CDEFCD95
:1017CB00756A02EE7872F6ED08F67F501218141255
:0617DB00196EEF20E0F999
:0117E10022E5
:10185600756A017F5012179312196EEF20E0F9781E
:0318660072E6FF28
:01186900225C
:101841001217C8E4FFFE0FBF00010EBE0FF8BFA0C4
:04185100F51218561E
:011855002270
:06154C00CBEFCBCAEECA92
:10155200300D03300E27756A03EA7872F6EB08F64F
:1015620008EDF67F5012181412196EEF20E0F9E41C
:0D157200FFFE0FBF00010EBE0FF8BFA0F579
:01157F002249
:10137D00753300753400753555E4F53212176FC3AA
:10138D0033CE33CED8F97C002532FFEC3EFEAB33A5
:10139D00AA34A935853282758300120660FD1215B7
:1013AD004C0532E532C3940640D27564007565066E
:0113BD00220D
:100F5D008E308F3112176FC333CE33CED8F925654E
:100F6D00FFE5643EFEEEC0E0EFC0E0E530FDD0E011
:100F7D00FFD0E0FE12154C0565E5657002056412A3
:100F8D00176FC333CE33CED8F92565FFE5643EFE2A
:100F9D00AD3112154C0565E565700205640559E521
:100FAD005970020558C3E5659440E56494004017F7
:100FBD00E4F564F5650563E56370020562AE62FFF5
:080FCD001217595002D20D2247
:10116B00E4F564F5657BFF7A19793A1215B4D20E62
:10117B00E4F53FF540AE3FAF401217594021E54033
:10118B00AE3F7806C333CE33CED8F9F5658E647D8A
:10119B0081FF12154C0540E54070DA053F80D6C241
:1011AB000E7BFF7A19793F1215B4E4F562F563F5FE
:0511BB0064F565C20DA2
:0111C000220C
:10111400E4F53FF540F541F542AE41AF42121759AF
:101124004044E5406481603EAF42AE411215E61290
:1011340018568F40E54064807022AF3F053FFCFDA8
:10114400FEFBFAF9120BBF7F2C12000EAE41AF4228
:10115400E4FCFDFBFAF9120BBF1219570542E542F4
:0611640070B7054180B3E5
:01116A002262
:0212B0008F3F6E
:1012B200E4F540F541F542F543AE42AF431217590A
:1012C2004030E5416481602AAF43AE421215E61216
:1012D20018568F41E541B4800FE540653F7007AF76
:1012E20043AE420215E605400543E54370CB054295
:0212F20080C7B3
:0112F40022D7
:10182B00121765E4F558F55912137D8562668563C9
:06183B00677F010210B0FE
:10147500856230856331E565456460080531E53190
:101485007002053085666285676312137D8530625B
:10149500853163AE30AF311217595007E4F562F567
:0814A50063D20D7F020210B0BA
:10186A00740478FF769612FF0322740078FF769646
:04187A0012FF032234
:03003300020DE8D3
:0D0DE800C0E0C0F0C083C082C0D075D0084C
:100DF500E5D954F8FF1208650E22080E22100E31AF
:100E0500180E4C200E33280E4C300E4E380E544022
:100E15000E4C480E6D500E8A5800000E98856DDAFE
:100E2500C2DDC2DC756B00756C008070800EE56AF2
:100E350070028056056CE56C7002056B1200268FFA
:100E4500DAC2DDC2DC80558016D2DDC2DC804DC23F
:100E5500DDC2DCE56A7004C2DA8041D2DA803DC2C7
:100E6500DDD2DC7568048034AFDA12192E056CE525
:100E75006C7002056BC2DDC2DCE56A7004C2DA8003
:100E85001BD2DA8017AFDA12192EC2DDD2DC7568F3
:0E0E9500028009756804C2DDC2DCD2DAC2DB5D
:0B0EA300D0D0D082D083D0F0D0E0325D
:1016440043910C43920CE4F5DBEF25E0F5DB300F1E
:101654000343DB0175DD2575DC2575D84453F8FE9D
:0916640053F7FEE4F568D2E82218
:10181400E56830E002FF22E4F569756803EF25E02E
:07182400F56DD2DD7F022209
:10179300E56830E002FF22E4F569156A756805EF34
:0B17A30025E04401F56DD2DD7F02223D
:06196E0020DBFDAF682242
:0D002600156AAF69056974722FF8E6FF22B4
:0C192E0074722569F8EFF60569156A224D
:0E18EC00E4F5847585FFF592F5A475A5FF223D
:07196000EE3395E0FDFC22CF
:10169500C20AC20CC209D2A2C2A0C2A1E4FDFF12B5
:1016A500173BE4FD7F0112173B7F081210B07F0442
:0316B5000210B070
:10173B00EF146011047016BD0104C2A78002D2A77A
:0E174B00A2A7920B22BD0103C2A622D2A622A3
:1010B000EF14B40800505C9010C575F003A4C5830C
:1010C00025F0C583730210DD0210E30210EA02105E
:1010D000F60210F80210F602110202110AD20A7585
:1010E000190122C20AA20B92A722D20C751A057D01
:1010F000017F0102173B8005C209C28722C209D2C3
:101100008722D209D28775180122C2A47F01121446
:04111000ADD2A42296
:1013FD00300A12D5190F30A707C2A775191E80051F
:10140D00D2A7751946E51AD39400400CD51A09C216
:10141D000CE4FD7F0112173B300911D5180E3087F2
:0D142D0006C28775180522D28775181E2289
:1016FB00C374039FFE1392A0EEA2E192A1AF80CF21
:0F170B005480CFED547FCF4FCF8F80C2A2D2A298
:01171A0022AC
:0615B4008B418A428943CD
:1015BA00E4FCCFECCF7D201216FB0CBC04F4E4FC57
:1015CA00AB41AA42A9438C82758300120660FD6072
:0B15DA000ACFECCF1216FB0CBC04E59E
:0115E50022E3
:040FD5008F828E83F6
:100FD900121960E47B0F7A27F9F8C31207EC500362
:100FE90090270FAF82AE831219607B197AFC79FFC3
:100FF90078FFD31207EC400390FC19E4F530741B19
:101009002530F8E4F60530E530B405F2AE83AF8259
:101019001219607B007A00791B120BBFE51E701A4A
:10102900753003741A2530F8E6FF741B2530F8C6AD
:10103900EFC6D530EE751B2080E27B007A00791B64
:031049000215B4D9
:1017E20046554C4C0050524F47005A4C4F47004D03
:0917F2004F44310076312E38001D
:030013000216DAF8
:1016DA00C0E0C0D075D01020060CAF8DEFAD8BF5F1
:1016EA005BEDF55CD206758D00758B00D0D0D0E02D
:0116FA0032BD
:0214AD008F406E
:1014AF00E4F541F542C3E5429540E54194005023F0
:1014BF00900000AF82AE83E4FCFD7B207A4EF9F8FA
:1014CF00D31207EC4003A380EA0542E54270D6052C
:0314DF004180D277
:0114E20022E7
:0E18FA007BFF7A1779E21215B47F0A0214AD53
:100036001218EC1219441216957F041214AD20976B
:10004600127BFF7A1779E71215B47F011212F5D2E7
:10005600AF80FE2096091203D812104C120A377A86
:100066001779EC1203CD7A1779F11203CD7BFF7A5B
:100076001779F61215B47F041214ADE4FF1212F5C7
:100086001203D87F011214AD12104C120011C212C5
:1000960012143A7F011214ADE4F55DF55E120012FA
:1000A600A2969200A2979201E4F52378A912084C31
:1000B60000000000E4F52478B112084CFFFFD8F1E7
:1000C60078A512084C00000000E4F55478AD12083B
:1000D6004C00000000C205C203C204E4F560F561ED
:1000E600F525F526F55BF55CC206F55FC20730120D
:1000F600FDC212300433A200309601B3400BA201B8
:10010600309701B340030201EA30961230970FC2CE
:1001160004E4F560F5617F041210B0E4F554A2968C
:100126009200A29792010201EA209605209702D238
:100136000830965D30975A300838C20878A51208FC
:1001460027EC4D4E4F78B1701312084C000000009A
:1001560078AD12082778A5120840801012084C00C6
:1001660000000078A512084C00000000D201D20061
:10017600802478BAE6601F0561E56170020560D3E8
:1001860094B8E560940B400ED2047F051210B0803F
:1001960005E4F560F561A200309601B3501DA29604
:1001A6009200309616200813E5546007E4F5547F54
:1001B6000680057554017F071210B0A20130970121
:1001C600B35021A297920130971A200817B2033034
:1001D600030F300D071218FAC203800812182B807D
:1001E600031214751203E520060302027BC2AFC296
:1001F60006D2AFE4855C2F855B2EF52DF52CAF2F4F
:10020600AE2EAD2DAC2C7B107A27F9F81206C18FD5
:100216002F8E2E8D2D8C2CE4FB7A90F9F812133943
:100226008F2F8E2E8D2D8C2C78C1E66009C374B865
:100236009FFF740B9EFEE55F14601624FE6020246B
:1002460003702FC3EF94B0EE9404500E755F0180D7
:1002560009D3EF9414EE9405401B755F038016C313
:10026600EF94B0EE9404500D755F01300307D2078A
:100276008003E4F55F0524E524C3940550030203D7
:10028600C7E4F524FB7A00792712166D8E288F298C
:10029600E527640260030203C778A9120833E8C0A1
:1002A600E0E9C0E0EAC0E0EBC0E078B9E6FDAF29DE
:1002B600AE28121264D0E0FBD0E0FAD0E0F9D0E02C
:1002C600F8EB2FFFEA3EFEE93DFDE83CFC78A9127B
:1002D60008400523E523C3940550030203C778A904
:1002E600120827E47B05FAF9F812133978A91208DF
:1002F6004078A912082778A5120833C3EF9BFFEEB2
:100306009AFEED99FDEC98FC78A912084078B11296
:10031600082778A9120833D31207EC400A78A912E5
:10032600082778B1120840E554600A78B3E6FE085B
:10033600E68E2AF52B78ABE6FE08E68E28F529E54B
:10034600546006AF2BAE2A8004AF29AE28120FD513
:1003560030035878B7E6FE08E6FFF47002EEF46064
:10036600180526E52670020525C39FE5259E401043
:10037600E4F525F526D2028007300704C207D2022B
:10038600300228C2027F031210B030050DE528FFA7
:1003960012000EAF29E52912000E200D09AF29AE75
:1003A60028120F5D80051218FAC20378A9120827D1
:1003B60078AD12084078A912084C00000000E4F558
:0703C600231213FD0200F4F5
:1003CD007BFF1215B47F041214AD22D2AF1217AEFB
:0803DD00C20F7F7012164422CA
:1016B800444C0021536967005A4C4F47004D4F4432
:1016C8003100312E38004D617220323420323030F2
:0216D8003400DC
:10121300AF38AE37AD36AC35EC4D4E4F22EF24FF31
:10122300F538EE34FFF537ED34FFF536EC34FFF5E2
:101233003522E475382075374EF536F53522E475D9
:101243003801F537F536F53522FDFCAB38AA37A959
:1012530036A835C30208027532007533007534B5FC
:011263002268
:1003E500121908EF70030206107F041210B0E4F52D
:1003F50054C204F560F561121776EF12086506041C
:1004050024060D2A056252042B6104996304EC65E8
:1004150005376C053D72053A7305667405D9760591
:10042500D178000006107BFF7A1679B81215B41240
:100435001235121908EF700A1212136005121220F4
:1004450080F012121370030206101217768F311204
:1004550012B0E4F538121245E47F06FE12124C5034
:100465000A1218568F3112061180ED1218568F3167
:10047500E53164806016E5316481601012000E126A
:1004850018568F3112000E7530018003E4F530E502
:100495003070D82212125A121241F531121213601D
:1004A50024121235121908EF700A12121360051280
:1004B500122080F0121213600312062A0531E5316D
:1004C500C3940E40D7121213601A78B5B6AB07085D
:1004D500B6CD0302060A7BFF7A1679BB1215B47FE7
:1004E5000A0214AD0205CEE4FFFE1217C8E4F53882
:1004F500121245E4FF7E0812124C50331218568F23
:1005050030E538540FFFE4FEFDFCFBFAF9F8C312A1
:100515000802700F121957AE37AF381218CD7F2069
:1005250012000EAF301217FB7F2012061180C40295
:100535000601B2052202111412125AE4F531AB324A
:100545000534E534AA337002053314F9120647FF62
:1005550012000E0531E531C3940E40E22243A20894
:1005650022753200753300753470121241F531125F
:1005750012136024121235121908EF700A121213A1
:10058500600512122080F0121213600312062A056C
:1005950031E531C3940240D7121213602CAE70AF0F
:1005A50071EE3395E0FDFC78AD120833C3EF9BF592
:1005B5003CEE9AF53BED99F53AEC98F539AF3C7878
:1005C500BFE53BF608EFF6803C0214E37F0412100A
:1005D500B002116B7A1679C012063E7A1679C512E9
:1005E500063E7F7612000E7BFF7A1679CA1218BA7C
:1005F5001219577BFF7A1679CE1218BA021957E4E9
:0B06050078BFF608F602161712151851
:100610002212000EE5382401F538E43537F537E4C9
:100620003536F536E43535F53522121776AB32AA74
:1006300033A934853182758300EF12069F227BFF38
:070640001218BA121957222B
:0A194400E4F5955396BF53A27F22ED
:10143A005389F0438901538FFE758C70E4F58A5302
:10144A00B8FD53B7FDD2A9D28C53890F4389905363
:10145A008FEFF58DF58B4391105392EF53B8F753F5
:0B146A00B7F7D2ABD28ED28AD2AA22F2
:03000B0002194E89
:09194E00D212758C70758A00320A
:03001B0002196760
:07196700758D00758B003245
:10187E000D0A003031323334353637383941424370
:04188E004445460087
:10189200AF53AB47AA48A949055322AF46AE45AD5F
:0418A20044AC4322ED
:1012F5005387BF75985053877FE4F5BABF010543FF
:10130500A240800353A2BFE4F5BD75BE30F5BF759D
:10131500BD035391FE4392014391025392FDC213C3
:1013250053B8EF53B7EF43B81078A3F618F678A47F
:04133500F6D2AC221E
:0300230002158043
:10158000C0E0C0D075D01030981E78A3E6C3940F89
:10159000501418E6062492F8A69978A30618E6C314
:1015A000941040027600C298309904C299C213D0B8
:0415B000D0D0E03285
:080003002013FDD2138F992296
:10171B0078A3E6D39400401508E6062492F8E6FF7A
:0F172B0078A31608E6C394104005E4F6227F0069
:01173A00228C
:03000E00020003EA
:101776007F207E4E78A3E67010D3EF9400EE94009F
:0C1786004007EF1F70EE1E80EB12171BD7
:011792002234
:1018BA00120647FF600C12000E740129F9E43AFA85
:0318CA0080EE228B
:0E19080078A3E6D3940040037F01227F0022E3
:1017FB00CEEFCEEE54F0C4540F90188193FF12002D
:09180B000EEE540F93FF02000ED3
:1018CD00CDEFCDCCEECCEEFF1217FBCFEDCF021747
:0118DD00FB0F
:091957007BFF7A18797E0218BAB0
:0E0BBF008F468E458D448C438B478A4889496A
:100BCD00E4F553EC4D4E4F7017E94A4B70057F30ED
:100BDD0002000E1218928F827583007430020CE29F
:100BED0012189FEC33502AE5494548454770077F59
:100BFD002D12000E800D1218928F82758300742DA8
:100C0D0012069F12189D1207DE8F468E458D448C5D
:100C1D0043755201754D00754CCA754B9A754A3B1B
:100C2D00E4FFFEFDFCAB4DAA4CA94BA84AD312081C
:100C3D00025003020CCD12189DA84A12074C8F5179
:100C4D008E508D4F8C4EEC4D4E4F7004E5527023EF
:100C5D00E5512430FFE54945484547700512000E22
:100C6D00800EAE531218948E82758300EF12069F7C
:100C7D00E4F552AF4DAE4CAD4BAC4AAB51AA50A9B9
:100C8D004FA84E1206C1C8ECC8C9EDC9CAEECAC3F9
:100C9D00E5469FF546E5459AF545E54499F544E564
:100CAD004398F543AF4DAE4CAD4BAC4AE47B0AFADD
:100CBD00F9F812074C8F4D8E4C8D4B8C4A020C2D32
:100CCD00E548454945476010AB47AA48A9498553B2
:080CDD0082758300E412069FFA
:010CE50022EC
:10088B000134C35001DBBF68028BBB800344B798B4
:10089B000407B3B004D5AFC805A9ABE00689A7F828
:1008AB000775A410086DA02809719C400A819858FF
:1008BB000B9F94700CCA90880DE98CF90E048CA0D8
:1008CB000EA88AAC0F4D88B80FF786C410A184D040
:1008DB00115182DC120580E812BB7EF413747D008B
:1008EB0014307B0C14F2791815B8772416807530F8
:1008FB00174B733C1819714818ED6F5419C46D6080
:10090B001AA16B6C1B7E69781C6167841D4A65900C
:10091B001E37639C1F2561A8201A5FB421125DC08E
:10092B00220D5BCC230E59D8241557E4251F55F007
:10093B00262F53FC27425208285B501429764E2051
:10094B002A9B4C2C2BC04A382CEE48442E1E46506A
:10095B002F55445C308F426831D1407433173E8041
:10096B0034633C8C35B13A98370938A4386636B0C5
:10097B0039C734BC3B2D32C83C9D30D43E0F2EE0E2
:10098B003F882CEC41062AF8428D29044418271085
:10099B0045AB251C4741232848E121344A861F409B
:1009AB004C311D4C4DE21B584F9C1964515D177017
:1009BB005323157C54EF138856C4119458A20FA0DF
:1009CB005A830DAC5C6D0BB85E6009C4605807D0E0
:1009DB00625A05DC646203E8667301F4688A0000FE
:1009EB006AA1FE0C6CB8FC186ECFFA2470E6F830D6
:1009FB0000000000000000000000000000000000EC
:100A0B0000000000000000000000000000000000DB
:100A1B0000000000000000000000000000000000CB
:0C0A2B00000000000000000000000000BF
:1013BE0075F004E537A4248BF582E5F03408F58347
:1013CE00E49322FE740193FF75F004E537A422F531
:1013DE0083C37401939FFFE4939EFEE4228F388EA5
:0F13EE00378D368C35228F348E338D328C3122F1
:1018A600C3EF9DEE9C400AD3EF9BEE9A50037F0157
:0418B600227F00226B
:040CE6008E358F3682
:100CEA00E4F5371213BEFC740193FD1213D6248F58
:100CFA00F582E5F03408F583E493FA740193FBAFC7
:100D0A0036AE351218A6EF7003020DD61213BE12B4
:100D1A0013D1248FF582E5F034081213DD8F3B8E50
:100D2A003AF539F5381213D62491F582E5F03408EC
:100D3A00F583E4931213D1248DF582E5F034081279
:100D4A0013DD8F3F8E3EF53DF53CAD3DAC3C1207C1
:100D5A00DE8F3F8E3E8D3D8C3CAE35AF36E4FCFDDA
:100D6A00EEC0E0EFC0E01213BEFE740193FBCAEEC0
:100D7A00CAD0E0FFD0E0FEC3EF9BFFEE9AFEED94EF
:100D8A0000FDEC9400FCAB3FAA3EA93DA83C12062C
:100D9A00C1AB3BAA3AA939A838121339C8ECC8C959
:100DAA00EDC9CAEECACBEFCB1213D6248DF582E574
:100DBA00F03408F583E493FE740193FFE4FCFDEB41
:100DCA002FFFEA3EFEED39FDEC38FC220537E53708
:0D0DDA00C3946A5003020CEDE4FFFEFDFC23
:010DE70022E9
:0100120022CB
:1011C1001213EBAB38AA37A936A835E8C0E078BDD1
:1011D100E6FE08E6FFE4FCFDD0E0F81206C11213BA
:1011E100EB780E1208131213EB78BFE6FE08E6FF48
:1011F100EE3395E0FDFCE5382FF538E5373EF53760
:10120100E5363DF536E5353CF535AF38AE37AD362B
:02121100FC22BD
:021264008D30CB
:10126600120CE61213F41211C11213F4E5301460D5
:101276001C14702DE47FE87E03FDFCAB34AA33A971
:1012860032A8311206C1E47BE87A0B800CAF34AE8B
:1012960033AD32AC31E47B03FAF9F8121339121389
:0912A600F4AF34AE33AD32AC31CB
:0112AF00221C
:10064700BB010689828A83E0225002E722BBFE02B1
:09065700E32289828A83E49322E4
:10066000BB010CE58229F582E5833AF583E022504F
:1006700006E92582F8E622BBFE06E92582F8E22299
:0D068000E58229F582E5833AF583E49322B3
:10068D00BB010689828A83F0225002F722BBFE014C
:02069D00F32246
:10069F00F8BB010DE58229F582E5833AF583E8F091
:1006AF00225006E92582C8F622BBFE05E92582C83D
:0206BF00F22225
:1006C100E88FF0A4CC8BF0A42CFCE98EF0A42CFCD8
:1006D1008AF0EDA42CFCEA8EF0A4CDA8F08BF0A456
:1006E1002DCC3825F0FDE98FF0A42CCD35F0FCEBB5
:1006F1008EF0A4FEA9F0EB8FF0A4CFC5F02ECD397A
:0F070100FEE43CFCEAA42DCE35F0FDE43CFC22E6
:1007100075F008758200EF2FFFEE33FECD33CDCCA0
:1007200033CCC58233C5829BED9AEC99E582984023
:100730000CF582EE9BFEED9AFDEC99FC0FD5F0D600
:10074000E4CEFBE4CDFAE4CCF9A88222B800C1B92A
:100750000059BA002DEC8BF084CFCECDFCE5F0CB68
:10076000F97818EF2FFFEE33FEED33FDEC33FCEBA1
:1007700033FB10D703994004EB99FB0FD8E5E4F95C
:10078000FA227818EF2FFFEE33FEED33FDEC33FC49
:10079000C933C910D7059BE99A4007EC9BFCE99A3D
:1007A000F90FD8E0E4C9FAE4CCFB2275F010EF2F82
:1007B000FFEE33FEED33FDCC33CCC833C810D70782
:1007C0009BEC9AE899400AED9BFDEC9AFCE899F8BD
:0E07D0000FD5F0DAE4CDFBE4CCFAE4C8F92250
:10133900C2D5E830E70FB2D5E4C39BFBE49AFAE4DF
:1013490099F9E498F8EC30E717B2D512136F120740
:101359004CE4C39BFBE49AFAE499F9E498F8800316
:1013690012074C30D50DE4C39FFFE49EFEE49DFDBA
:04137900E49CFC22D2
:0E07DE00C3E49FFFE49EFEE49DFDE49CFC222C
:1007EC00EB9FF5F0EA9E42F0E99D42F0EC6480C884
:0607FC0064809845F02224
:10080200EB9FF5F0EA9E42F0E99D42F0E89C45F04C
:0108120022C3
:10081300E86010ECA2E713FCED13FDEE13FEEF13FB
:04082300FFD8F022E8
:0C082700E6FC08E6FD08E6FE08E6FF22FD
:0D083300E6FB08E6F908E6FA08E6CBF82235
:0C084000ECF608EDF608EEF608EFF622E4
:10084C00D083D082E493F608740193F60874029373
:09085C00F608740393F6740473AA
:10086500D083D082F8E4937012740193700DA3A322
:1008750093F8740193F5828883E473740293686036
:06088500EFA3A3A380DF36
:00000001FF
